:020000040000FA
:04000000A0EF3FF03E
:087F3800000000000000000041
:107F4000240EAC6E0A0EAF6E900EAB6E46D8C10812
:107F500053E1550EAD6E4B0EAD6E006A3ED8F86E15
:107F6000076E3BD8F76EA96E38D8F66EA86E35D876
:107F7000016E012A00EE09F0F56E2FD8EC6E012E8D
:107F8000FBD700661FD007AC03D0040E1ED818D054
:107F900007AE04D00C00C40E18D812D0940E15D819
:107FA0000A00020E056E00EE0AF0200E066EEE507C
:107FB000F56E0F00062EFBD7840E07D8052EF5D7D9
:107FC000A694C9D74E0EAD6EC8D7A66E550EA76E35
:107FD000AA0EA76EA682000012000B0E026E036AA4
:107FE000046A9EAA03D0AE5000261200042EF9D7D0
:0C7FF000032EF6D7022EF3D7AB9E9ED7CF
:020000040030CA
:0E000000E43CC6EEFFF9BAFFFFFFFFFFFFFF73
:00000001FF
